:100000007029FF3FFF3FFF3F03138312A0018118B8
:100010000728811C092807130430A000231814287E
:100020008118102807131728811814280717A30C04
:1000300023181E28811C1A2807132128811C1E281A
:100040000717A30CA00B0E288118242807170800F7
:100050000030031783168C180130F1007108013A43
:100060000319282803138312210803178D00031393
:10007000220803178C0083160C15031783165530BE
:100080008D00AA308D008C140C11080099300313D8
:100090008312A300042024087F3C031851287F30DA
:1000A000A4002408A300042025087F3C03185A2834
:1000B0007F30A5002508A300042008000313831245
:1000C000210803178D0083160C1483120C080313E8
:1000D000A20008000130031383120705F100710824
:1000E000003A031DC028003087180130F100710864
:1000F000003A031DC0282608003A031D812828085D
:10010000A7002608013A031D87282808A900260809
:10011000023A031D8D282808AA002608033A031D69
:1001200093282808AB002608043A031D99282808BC
:10013000AC002608053A031D9F282808AD002608B4
:10014000063A031DA5282808AE002608073A031D15
:10015000AB282808AF002608083A031DB128280854
:10016000B0002608093A031DB7282808B10028085E
:10017000A5002608203FA1002808A2002820662903
:100180000130031383120705F1007108003A031DC3
:100190001429A403173024020318D0281730A40010
:1001A0002608A1002408A200282003138312260891
:1001B000003A031DDD282408B2002608013A031D79
:1001C000E3282408B3002608023A031DE92824087E
:1001D000B4002608033A031DEF282408B5002608BA
:1001E000043A031DF5282408B6002608053A031D25
:1001F000FB282408B7002608063A031D0129240815
:10020000B8002608073A031D07292408B900260864
:10021000083A031D0D292408BA002608093A031DCF
:1002200013292408BB006629003087180130F1002B
:100230007108003A031D6629A40A2408623C0318C9
:1002400023296230A4002608A1002408A200282047
:10025000031383122608003A031D30292408B20034
:100260002608013A031D36292408B3002608023A5D
:10027000031D3C292408B4002608033A031D422923
:100280002408B5002608043A031D48292408B600AE
:100290002608053A031D4E292408B7002608063A09
:1002A000031D54292408B8002608073A031D5A29BB
:1002B0002408B9002608083A031D60292408BA005A
:1002C0002608093A031D66292408BB00031383127C
:1002D0002508003A031D6E292808A50046200800BD
:1002E0008130031383129F000E3083169F00831208
:1002F000850101308316850083128601FF30831645
:100300008600831287010F30831687008B0104302B
:10031000810003178C0103138312900187010717D3
:100320006430A800A1015E202208B2002030A1079D
:100330005E202208A7000130A1005E202208B30041
:100340002030A1075E202208A9000230A1005E2013
:100350002208B4002030A1075E202208AA00033042
:10036000A1005E202208B5002030A1075E202208EF
:10037000AB000430A1005E202208B6002030A107A7
:100380005E202208AC000530A1005E202208B700E4
:100390002030A1075E202208AD000630A1005E20BB
:1003A0002208B8002030A1075E202208AE000730E6
:1003B000A1005E202208B9002030A1075E2022089B
:1003C000AF000830A1005E202208BA002030A1074B
:1003D0005E202208B0000930A1005E202208BB0088
:1003E0002030A1075E202208B100C830BC00C83010
:1003F000BD00C830BE00C830BF00C830C000C83023
:10040000C100C830C200C830C300C830C400C83002
:10041000C50081010B113C08003A031D1E2A013062
:100420000605F1007108003A031D1E2A1530BC00B4
:10043000A6013208A4002708A5006A203D08003A5A
:10044000031D332A003086180130F1007108003A8C
:10045000031D332A1530BD000130A6003308A40067
:100460002908A5006A203E08003A031D482A0030EA
:1004700006190130F1007108003A031D482A1530B1
:10048000BE000230A6003408A4002A08A5006A2095
:100490003F08003A031D5D2A003086190130F10043
:1004A0007108003A031D5D2A1530BF000330A60015
:1004B0003508A4002B08A5006A204008003A031D57
:1004C000722A0030061A0130F1007108003A031D4B
:1004D000722A1530C0000430A6003608A4002C088B
:1004E000A5006A204108003A031D872A0030861AB9
:1004F0000130F1007108003A031D872A1530C10050
:100500000530A6003708A4002D08A5006A2042087F
:10051000003A031D9C2A0030061B0130F1007108CF
:10052000003A031D9C2A1530C2000630A600380888
:10053000A4002E08A5006A204308003A031DB12A32
:100540000030861B0130F1007108003A031DB12A0A
:100550001530C3000730A6003908A4002F08A500F5
:100560006A204408003A031DC62A003007190130EA
:10057000F1007108003A031DC62A1530C400083086
:10058000A6003A08A4003008A5006A204508003AF1
:10059000031DDB2A003087190130F1007108003A91
:1005A000031DDB2A1530C5000930A6003B08A40056
:1005B0003108A5006A2000300B190130F1007108E4
:1005C000013A031DCB2B0B1187123C08003C03188A
:1005D000F82ABC033C08003A031DF72A013006053F
:1005E000F1007108003A031DF72A0530BC00871698
:1005F0003D08003C03180C2BBD033D08003A031DC9
:100600000B2B003086180130F1007108003A031DF1
:100610000B2B0530BD0087163E08003C0318202B2D
:10062000BE033E08003A031D1F2B0030061901309F
:10063000F1007108003A031D1F2B0530BE0087161C
:100640003F08003C0318342BBF033F08003A031D4A
:10065000332B003086190130F1007108003A031D78
:10066000332B0530BF0087164008003C0318482B89
:10067000C0034008003A031D472B0030061A013022
:10068000F1007108003A031D472B0530C0008716A2
:100690004108003C03185C2BC1034108003A031DCC
:1006A0005B2B0030861A0130F1007108003A031DFF
:1006B0005B2B0530C10087164208003C0318702BE5
:1006C000C2034208003A031D6F2B0030061B0130A5
:1006D000F1007108003A031D6F2B0530C200871628
:1006E0004308003C0318842BC3034308003A031D4E
:1006F000832B0030861B0130F1007108003A031D86
:10070000832B0530C30087164408003C0318982B40
:10071000C4034408003A031D972B00300719013029
:10072000F1007108003A031D972B0530C4008716AD
:100730004508003C0318AC2BC5034508003A031DCF
:10074000AB2B003087190130F1007108003A031D0E
:10075000AB2B0530C5008716C60A4608093A031DAB
:10076000B22B1F150A304602031CCB2B1E08A80013
:100770000130F4002808F00074080319C32BF00CB2
:10078000F013FF3FBD2B7008A8000530700203185E
:10079000CA2BA801C6010B2ACC2BFF3FFF3FFF3F0E
:02400E00723FFF
:00000001FF
